 JNIreferences

 Timestamp is f85bf050 (reproducible build file hash)

 Preferred load address is 0000000180000000

 Start         Length     Name                   Class
 0001:00000000 00001640H .text$mn                CODE
 0001:00001640 00000036H .text$mn$00             CODE
 0001:00001676 00000092H .text$x                 CODE
 0002:00000000 00000150H .idata$5                DATA
 0002:00000150 00000038H .00cfg                  DATA
 0002:00000188 00000008H .CRT$XCA                DATA
 0002:00000190 00000008H .CRT$XCZ                DATA
 0002:00000198 00000008H .CRT$XIA                DATA
 0002:000001a0 00000008H .CRT$XIZ                DATA
 0002:000001a8 00000008H .CRT$XPA                DATA
 0002:000001b0 00000008H .CRT$XPZ                DATA
 0002:000001b8 00000008H .CRT$XTA                DATA
 0002:000001c0 00000010H .CRT$XTZ                DATA
 0002:000001c8 00000000H .gehcont$y              DATA
 0002:000001c8 00000000H .gfids$y                DATA
 0002:000001d0 00000730H .rdata                  DATA
 0002:00000900 00000000H .rdata$CastGuardVftablesA DATA
 0002:00000900 00000000H .rdata$CastGuardVftablesC DATA
 0002:00000900 00000064H .rdata$voltmd           DATA
 0002:00000964 0000029cH .rdata$zzzdbg           DATA
 0002:00000c00 00000008H .rtc$IAA                DATA
 0002:00000c08 00000008H .rtc$IZZ                DATA
 0002:00000c10 00000008H .rtc$TAA                DATA
 0002:00000c18 00000008H .rtc$TZZ                DATA
 0002:00000c20 00000200H .xdata                  DATA
 0002:00000e20 000001a0H .edata                  DATA
 0002:00000fc0 00000078H .idata$2                DATA
 0002:00001038 00000018H .idata$3                DATA
 0002:00001050 00000150H .idata$4                DATA
 0002:000011a0 0000037eH .idata$6                DATA
 0003:00000000 00000040H .data                   DATA
 0003:00000040 00000620H .bss                    DATA
 0004:00000000 00000258H .pdata                  DATA

  Address         Publics by Value              Rva+Base               Lib:Object

 0000:00000000       __AbsoluteZero             0000000000000000     <absolute>
 0000:00000000       ___safe_se_handler_count   0000000000000000     <absolute>
 0000:00000000       ___safe_se_handler_table   0000000000000000     <absolute>
 0000:00000000       __arm64x_extra_rfe_table   0000000000000000     <absolute>
 0000:00000000       __arm64x_extra_rfe_table_size 0000000000000000     <absolute>
 0000:00000000       __arm64x_native_entrypoint 0000000000000000     <absolute>
 0000:00000000       __arm64x_redirection_metadata 0000000000000000     <absolute>
 0000:00000000       __arm64x_redirection_metadata_count 0000000000000000     <absolute>
 0000:00000000       __dynamic_value_reloc_table 0000000000000000     <absolute>
 0000:00000000       __enclave_config           0000000000000000     <absolute>
 0000:00000000       __guard_check_icall_a64n_fptr 0000000000000000     <absolute>
 0000:00000000       __guard_eh_cont_count      0000000000000000     <absolute>
 0000:00000000       __guard_eh_cont_table      0000000000000000     <absolute>
 0000:00000000       __guard_fids_count         0000000000000000     <absolute>
 0000:00000000       __guard_fids_table         0000000000000000     <absolute>
 0000:00000000       __guard_iat_count          0000000000000000     <absolute>
 0000:00000000       __guard_iat_table          0000000000000000     <absolute>
 0000:00000000       __guard_longjmp_count      0000000000000000     <absolute>
 0000:00000000       __guard_longjmp_table      0000000000000000     <absolute>
 0000:00000000       __hybrid_auxiliary_iat     0000000000000000     <absolute>
 0000:00000000       __hybrid_auxiliary_iat_copy 0000000000000000     <absolute>
 0000:00000000       __hybrid_code_map          0000000000000000     <absolute>
 0000:00000000       __hybrid_code_map_count    0000000000000000     <absolute>
 0000:00000000       __x64_code_ranges_to_entry_points 0000000000000000     <absolute>
 0000:00000000       __x64_code_ranges_to_entry_points_count 0000000000000000     <absolute>
 0000:00000100       __guard_flags              0000000000000100     <absolute>
 0000:00000000       __ImageBase                0000000180000000     <linker-defined>
 0001:00000000       ?CallVoidMethod@JNIEnv_@@QEAAXPEAV_jobject@@PEAU_jmethodID@@ZZ 0000000180001000 f i libJNIreferences.obj
 0001:00000024       Java_nsk_share_ReferringObject_createJNIGlobalReferenceNative 0000000180001024 f   libJNIreferences.obj
 0001:00000144       Java_nsk_share_ReferringObject_createJNILocalReferenceNative 0000000180001144 f   libJNIreferences.obj
 0001:0000024c       Java_nsk_share_ReferringObject_createJNIWeakReferenceNative 000000018000124c f   libJNIreferences.obj
 0001:00000374       Java_nsk_share_ReferringObject_deleteJNIGlobalReferenceNative 0000000180001374 f   libJNIreferences.obj
 0001:00000408       Java_nsk_share_ReferringObject_deleteJNIWeakReferenceNative 0000000180001408 f   libJNIreferences.obj
 0001:000004f8       __local_stdio_printf_options 00000001800014f8 f i libJNIreferences.obj
 0001:00000530       fprintf                    0000000180001530 f i libJNIreferences.obj
 0001:00000574       nsk_lcomplain              0000000180001574 f   libJNIreferences.obj
 0001:00000594       nsk_lvcomplain             0000000180001594 f   libJNIreferences.obj
 0001:0000074c       nsk_printf                 000000018000174c f   libJNIreferences.obj
 0001:00000774       nsk_vprintf                0000000180001774 f   libJNIreferences.obj
 0001:00000828       printf                     0000000180001828 f i libJNIreferences.obj
 0001:00000878       __raise_securityfailure    0000000180001878 f   MSVCRT:gs_report.obj
 0001:000008ac       __report_gsfailure         00000001800018ac f   MSVCRT:gs_report.obj
 0001:000009f4       __GSHandlerCheck           00000001800019f4 f   MSVCRT:gshandler.obj
 0001:00000a14       __GSHandlerCheckCommon     0000000180001a14 f   MSVCRT:gshandler.obj
 0001:00000a80       __security_check_cookie    0000000180001a80 f   MSVCRT:amdsecgs.obj
 0001:00000dc0       _DllMainCRTStartup         0000000180001dc0 f   MSVCRT:dll_dllmain.obj
 0001:00000e00       __security_init_cookie     0000000180001e00 f   MSVCRT:gs_support.obj
 0001:00000eac       DllMain                    0000000180001eac f   MSVCRT:dll_dllmain_stub.obj
 0001:00000ed0       ?__scrt_initialize_type_info@@YAXXZ 0000000180001ed0 f   MSVCRT:tncleanup.obj
 0001:00000ee0       ?__scrt_uninitialize_type_info@@YAXXZ 0000000180001ee0 f   MSVCRT:tncleanup.obj
 0001:00000eec       __local_stdio_scanf_options 0000000180001eec f i MSVCRT:default_local_stdio_options.obj
 0001:00000ef4       __scrt_initialize_default_local_stdio_options 0000000180001ef4 f   MSVCRT:default_local_stdio_options.obj
 0001:00000f10       __scrt_acquire_startup_lock 0000000180001f10 f   MSVCRT:utility.obj
 0001:00000f4c       __scrt_dllmain_after_initialize_c 0000000180001f4c f   MSVCRT:utility.obj
 0001:00000f80       __scrt_dllmain_before_initialize_c 0000000180001f80 f   MSVCRT:utility.obj
 0001:00000f98       __scrt_dllmain_crt_thread_attach 0000000180001f98 f   MSVCRT:utility.obj
 0001:00000fc0       __scrt_dllmain_crt_thread_detach 0000000180001fc0 f   MSVCRT:utility.obj
 0001:00000fd8       __scrt_dllmain_exception_filter 0000000180001fd8 f   MSVCRT:utility.obj
 0001:00001038       __scrt_dllmain_uninitialize_c 0000000180002038 f   MSVCRT:utility.obj
 0001:00001068       __scrt_dllmain_uninitialize_critical 0000000180002068 f   MSVCRT:utility.obj
 0001:0000107c       __scrt_initialize_crt      000000018000207c f   MSVCRT:utility.obj
 0001:000010c8       __scrt_initialize_onexit_tables 00000001800020c8 f   MSVCRT:utility.obj
 0001:00001154       __scrt_is_nonwritable_in_current_image 0000000180002154 f   MSVCRT:utility.obj
 0001:000011ec       __scrt_release_startup_lock 00000001800021ec f   MSVCRT:utility.obj
 0001:00001210       __scrt_uninitialize_crt    0000000180002210 f   MSVCRT:utility.obj
 0001:0000123c       __scrt_get_dyn_tls_init_callback 000000018000223c f   MSVCRT:dyn_tls_init.obj
 0001:00001244       __crt_debugger_hook        0000000180002244 f   MSVCRT:utility_desktop.obj
 0001:0000124c       __scrt_fastfail            000000018000224c f   MSVCRT:utility_desktop.obj
 0001:00001398       _RTC_Initialize            0000000180002398 f   MSVCRT:initsect.obj
 0001:000013d4       _RTC_Terminate             00000001800023d4 f   MSVCRT:initsect.obj
 0001:00001410       _guard_check_icall_nop     0000000180002410 f i MSVCRT:guard_support.obj
 0001:00001414       __isa_available_init       0000000180002414 f   MSVCRT:cpu_disp.obj
 0001:000015c0       _get_startup_argv_mode     00000001800025c0 f   MSVCRT:argv_mode.obj
 0001:000015c8       __scrt_is_ucrt_dll_in_use  00000001800025c8 f   MSVCRT:ucrt_detection.obj
 0001:000015e0       strchr                     00000001800025e0 f   vcruntime:VCRUNTIME140.dll
 0001:000015e6       memset                     00000001800025e6 f   vcruntime:VCRUNTIME140.dll
 0001:000015ec       __C_specific_handler       00000001800025ec f   vcruntime:VCRUNTIME140.dll
 0001:000015f2       __std_type_info_destroy_list 00000001800025f2 f   vcruntime:VCRUNTIME140.dll
 0001:000015f8       strlen                     00000001800025f8 f   ucrt:api-ms-win-crt-string-l1-1-0.dll
 0001:000015fe       _initterm                  00000001800025fe f   ucrt:api-ms-win-crt-runtime-l1-1-0.dll
 0001:00001604       _initterm_e                0000000180002604 f   ucrt:api-ms-win-crt-runtime-l1-1-0.dll
 0001:0000160a       _seh_filter_dll            000000018000260a f   ucrt:api-ms-win-crt-runtime-l1-1-0.dll
 0001:00001610       _configure_narrow_argv     0000000180002610 f   ucrt:api-ms-win-crt-runtime-l1-1-0.dll
 0001:00001616       _initialize_narrow_environment 0000000180002616 f   ucrt:api-ms-win-crt-runtime-l1-1-0.dll
 0001:0000161c       _initialize_onexit_table   000000018000261c f   ucrt:api-ms-win-crt-runtime-l1-1-0.dll
 0001:00001622       _execute_onexit_table      0000000180002622 f   ucrt:api-ms-win-crt-runtime-l1-1-0.dll
 0001:00001628       _cexit                     0000000180002628 f   ucrt:api-ms-win-crt-runtime-l1-1-0.dll
 0001:00001630       __acrt_initialize          0000000180002630 f   MSVCRT:ucrt_stubs.obj
 0001:00001630       __acrt_thread_attach       0000000180002630 f   MSVCRT:ucrt_stubs.obj
 0001:00001630       __acrt_thread_detach       0000000180002630 f   MSVCRT:ucrt_stubs.obj
 0001:00001630       __acrt_uninitialize        0000000180002630 f   MSVCRT:ucrt_stubs.obj
 0001:00001630       __acrt_uninitialize_critical 0000000180002630 f   MSVCRT:ucrt_stubs.obj
 0001:00001630       __scrt_stub_for_acrt_initialize 0000000180002630 f   MSVCRT:ucrt_stubs.obj
 0001:00001630       __scrt_stub_for_acrt_thread_attach 0000000180002630 f   MSVCRT:ucrt_stubs.obj
 0001:00001630       __scrt_stub_for_acrt_thread_detach 0000000180002630 f   MSVCRT:ucrt_stubs.obj
 0001:00001630       __scrt_stub_for_acrt_uninitialize 0000000180002630 f   MSVCRT:ucrt_stubs.obj
 0001:00001630       __scrt_stub_for_acrt_uninitialize_critical 0000000180002630 f   MSVCRT:ucrt_stubs.obj
 0001:00001630       __vcrt_initialize          0000000180002630 f   MSVCRT:ucrt_stubs.obj
 0001:00001630       __vcrt_thread_attach       0000000180002630 f   MSVCRT:ucrt_stubs.obj
 0001:00001630       __vcrt_thread_detach       0000000180002630 f   MSVCRT:ucrt_stubs.obj
 0001:00001630       __vcrt_uninitialize        0000000180002630 f   MSVCRT:ucrt_stubs.obj
 0001:00001630       __vcrt_uninitialize_critical 0000000180002630 f   MSVCRT:ucrt_stubs.obj
 0001:00001634       __scrt_stub_for_is_c_termination_complete 0000000180002634 f   MSVCRT:ucrt_stubs.obj
 0001:00001634       _is_c_termination_complete 0000000180002634 f   MSVCRT:ucrt_stubs.obj
 0001:00001637       memcpy                     0000000180002637 f   vcruntime:VCRUNTIME140.dll
 0001:00001650       _guard_dispatch_icall_nop  0000000180002650 f   MSVCRT:guard_dispatch.obj
 0001:00001670       _guard_xfg_dispatch_icall_nop 0000000180002670 f   MSVCRT:guard_xfg_dispatch.obj
 0002:00000000       __imp_RtlCaptureContext    0000000180003000     kernel32:KERNEL32.dll
 0002:00000008       __imp_RtlLookupFunctionEntry 0000000180003008     kernel32:KERNEL32.dll
 0002:00000010       __imp_RtlVirtualUnwind     0000000180003010     kernel32:KERNEL32.dll
 0002:00000018       __imp_UnhandledExceptionFilter 0000000180003018     kernel32:KERNEL32.dll
 0002:00000020       __imp_SetUnhandledExceptionFilter 0000000180003020     kernel32:KERNEL32.dll
 0002:00000028       __imp_GetCurrentProcess    0000000180003028     kernel32:KERNEL32.dll
 0002:00000030       __imp_TerminateProcess     0000000180003030     kernel32:KERNEL32.dll
 0002:00000038       __imp_IsProcessorFeaturePresent 0000000180003038     kernel32:KERNEL32.dll
 0002:00000040       __imp_QueryPerformanceCounter 0000000180003040     kernel32:KERNEL32.dll
 0002:00000048       __imp_GetCurrentProcessId  0000000180003048     kernel32:KERNEL32.dll
 0002:00000050       __imp_GetCurrentThreadId   0000000180003050     kernel32:KERNEL32.dll
 0002:00000058       __imp_GetSystemTimeAsFileTime 0000000180003058     kernel32:KERNEL32.dll
 0002:00000060       __imp_DisableThreadLibraryCalls 0000000180003060     kernel32:KERNEL32.dll
 0002:00000068       __imp_InitializeSListHead  0000000180003068     kernel32:KERNEL32.dll
 0002:00000070       __imp_IsDebuggerPresent    0000000180003070     kernel32:KERNEL32.dll
 0002:00000078       \177KERNEL32_NULL_THUNK_DATA 0000000180003078     kernel32:KERNEL32.dll
 0002:00000080       __imp_strchr               0000000180003080     vcruntime:VCRUNTIME140.dll
 0002:00000088       __imp_memset               0000000180003088     vcruntime:VCRUNTIME140.dll
 0002:00000090       __imp___C_specific_handler 0000000180003090     vcruntime:VCRUNTIME140.dll
 0002:00000098       __imp___std_type_info_destroy_list 0000000180003098     vcruntime:VCRUNTIME140.dll
 0002:000000a0       __imp_memcpy               00000001800030a0     vcruntime:VCRUNTIME140.dll
 0002:000000a8       \177VCRUNTIME140_NULL_THUNK_DATA 00000001800030a8     vcruntime:VCRUNTIME140.dll
 0002:000000b0       __imp_malloc               00000001800030b0     ucrt:api-ms-win-crt-heap-l1-1-0.dll
 0002:000000b8       \177api-ms-win-crt-heap-l1-1-0_NULL_THUNK_DATA 00000001800030b8     ucrt:api-ms-win-crt-heap-l1-1-0.dll
 0002:000000c0       __imp__execute_onexit_table 00000001800030c0     ucrt:api-ms-win-crt-runtime-l1-1-0.dll
 0002:000000c8       __imp__errno               00000001800030c8     ucrt:api-ms-win-crt-runtime-l1-1-0.dll
 0002:000000d0       __imp__configure_narrow_argv 00000001800030d0     ucrt:api-ms-win-crt-runtime-l1-1-0.dll
 0002:000000d8       __imp__cexit               00000001800030d8     ucrt:api-ms-win-crt-runtime-l1-1-0.dll
 0002:000000e0       __imp__initterm            00000001800030e0     ucrt:api-ms-win-crt-runtime-l1-1-0.dll
 0002:000000e8       __imp__initterm_e          00000001800030e8     ucrt:api-ms-win-crt-runtime-l1-1-0.dll
 0002:000000f0       __imp__seh_filter_dll      00000001800030f0     ucrt:api-ms-win-crt-runtime-l1-1-0.dll
 0002:000000f8       __imp__initialize_onexit_table 00000001800030f8     ucrt:api-ms-win-crt-runtime-l1-1-0.dll
 0002:00000100       __imp__initialize_narrow_environment 0000000180003100     ucrt:api-ms-win-crt-runtime-l1-1-0.dll
 0002:00000108       \177api-ms-win-crt-runtime-l1-1-0_NULL_THUNK_DATA 0000000180003108     ucrt:api-ms-win-crt-runtime-l1-1-0.dll
 0002:00000110       __imp___stdio_common_vfprintf 0000000180003110     ucrt:api-ms-win-crt-stdio-l1-1-0.dll
 0002:00000118       __imp___stdio_common_vsprintf 0000000180003118     ucrt:api-ms-win-crt-stdio-l1-1-0.dll
 0002:00000120       __imp___acrt_iob_func      0000000180003120     ucrt:api-ms-win-crt-stdio-l1-1-0.dll
 0002:00000128       __imp_fflush               0000000180003128     ucrt:api-ms-win-crt-stdio-l1-1-0.dll
 0002:00000130       \177api-ms-win-crt-stdio-l1-1-0_NULL_THUNK_DATA 0000000180003130     ucrt:api-ms-win-crt-stdio-l1-1-0.dll
 0002:00000138       __imp_strlen               0000000180003138     ucrt:api-ms-win-crt-string-l1-1-0.dll
 0002:00000140       __imp_strncpy              0000000180003140     ucrt:api-ms-win-crt-string-l1-1-0.dll
 0002:00000148       \177api-ms-win-crt-string-l1-1-0_NULL_THUNK_DATA 0000000180003148     ucrt:api-ms-win-crt-string-l1-1-0.dll
 0002:00000150       __guard_check_icall_fptr   0000000180003150     MSVCRT:guard_support.obj
 0002:00000158       __guard_xfg_check_icall_fptr 0000000180003158     MSVCRT:guard_support.obj
 0002:00000160       __guard_dispatch_icall_fptr 0000000180003160     MSVCRT:guard_support.obj
 0002:00000168       __guard_xfg_dispatch_icall_fptr 0000000180003168     MSVCRT:guard_support.obj
 0002:00000170       __guard_xfg_table_dispatch_icall_fptr 0000000180003170     MSVCRT:guard_support.obj
 0002:00000178       __castguard_check_failure_os_handled_fptr 0000000180003178     MSVCRT:guard_support.obj
 0002:00000180       __guard_memcpy_fptr        0000000180003180     vcruntime:softmemtag.obj
 0002:00000188       __xc_a                     0000000180003188     MSVCRT:initializers.obj
 0002:00000190       __xc_z                     0000000180003190     MSVCRT:initializers.obj
 0002:00000198       __xi_a                     0000000180003198     MSVCRT:initializers.obj
 0002:000001a0       __xi_z                     00000001800031a0     MSVCRT:initializers.obj
 0002:000001a8       __xp_a                     00000001800031a8     MSVCRT:initializers.obj
 0002:000001b0       __xp_z                     00000001800031b0     MSVCRT:initializers.obj
 0002:000001b8       __xt_a                     00000001800031b8     MSVCRT:initializers.obj
 0002:000001c0       __xt_z                     00000001800031c0     MSVCRT:initializers.obj
 0002:000001d0       ??_C@_0BE@MIAHPFIA@malloc?5return?5null?6@ 00000001800031d0     libJNIreferences.obj
 0002:000001f0       ??_C@_0EA@IDOBAIL@s?2test?2hotspot?2jtreg?2vmTestbase@ 00000001800031f0     libJNIreferences.obj
 0002:00000230       ??_C@_0BK@DNFOEBEO@NewGlobalRef?5return?5null?6@ 0000000180003230     libJNIreferences.obj
 0002:00000250       ??_C@_0BJ@GGABHAHL@NewGlobalRef?5return?5null@ 0000000180003250     libJNIreferences.obj
 0002:00000270       ??_C@_0BH@IHJOPPGD@nsk?1share?1TestJNIError@ 0000000180003270     libJNIreferences.obj
 0002:00000288       ??_C@_0DN@DNGFLNOG@globalReferences?$FL?$CFd?$FN?5?$DN?5null?0?5po@ 0000000180003288     libJNIreferences.obj
 0002:000002d0       ??_C@_0EN@CMCIPPIF@Requested?5globalReferences?$FL?$FN?5el@ 00000001800032d0     libJNIreferences.obj
 0002:00000320       ??_C@_0BC@JDKHJCGI@nsk?1share?1TestBug@ 0000000180003320     libJNIreferences.obj
 0002:00000338       ??_C@_0BJ@DEKHJNIG@NewLocalRef?5return?5null?6@ 0000000180003338     libJNIreferences.obj
 0002:00000358       ??_C@_0BI@CJJBJDHH@NewLocalRef?5return?5null@ 0000000180003358     libJNIreferences.obj
 0002:00000370       ??_C@_03GAEACAIP@?$CI?$CJV@ 0000000180003370     libJNIreferences.obj
 0002:00000374       ??_C@_06BNCCALCL@unlock@   0000000180003374     libJNIreferences.obj
 0002:00000380       ??_C@_07NCNNHHFL@waitFor@  0000000180003380     libJNIreferences.obj
 0002:00000388       ??_C@_0BO@NCJJJNKP@NewWeakGlobalRef?5return?5null?6@ 0000000180003388     libJNIreferences.obj
 0002:000003a8       ??_C@_0BN@HEMNLLDI@NewWeakGlobalRef?5return?5null@ 00000001800033a8     libJNIreferences.obj
 0002:000003c8       ??_C@_0DL@BLJLHPON@weakReferences?$FL?$CFd?$FN?5?$DN?5null?0?5poss@ 00000001800033c8     libJNIreferences.obj
 0002:00000410       ??_C@_0EL@GCICLILG@Requested?5weakReferences?$FL?$FN?5elem@ 0000000180003410     libJNIreferences.obj
 0002:00000460       ??_C@_0CI@NANIDFCI@TEST?5BUG?3?5Weak?5reference?5was?5co@ 0000000180003460     libJNIreferences.obj
 0002:00000488       ??_C@_0CH@FIPGDGPL@TEST?5BUG?3?5Weak?5reference?5was?5co@ 0000000180003488     libJNIreferences.obj
 0002:000004b0       ??_C@_0JI@HLPECLFI@?$CD?5?4?4?4?6?$CD?5ERROR?3?5too?5many?5complai@ 00000001800034b0     libJNIreferences.obj
 0002:00000550       ??_C@_0ED@JNEKCCOB@The?5following?5fake?5exception?5st@ 0000000180003550     libJNIreferences.obj
 0002:00000598       ??_C@_0CN@FCNMDFBH@nsk?4share?4Fake_Exception_for_RU@ 0000000180003598     libJNIreferences.obj
 0002:000005c8       ??_C@_08PGFFNAEI@?$CI?$CFs?3?$CFd?$CJ?5@ 00000001800035c8     libJNIreferences.obj
 0002:000005d8       ??_C@_0DP@IENMAEGI@s?2test?2hotspot?2jtreg?2vmTestbase@ 00000001800035d8     libJNIreferences.obj
 0002:00000618       ??_C@_0BL@NDJLFFJB@?7at?5nsk_lvcomplain?$CI?$CFs?3?$CFd?$CJ?6@ 0000000180003618     libJNIreferences.obj
 0002:00000638       ??_C@_0BC@JOOKAFKF@?$CD?5ERROR?3?5?$CFs?0?5?$CFd?3?5@ 0000000180003638     libJNIreferences.obj
 0002:00000650       ??_C@_09KJEAHMEH@?$CD?5ERROR?3?5@ 0000000180003650     libJNIreferences.obj
 0002:00000660       ??_C@_0CO@LGONDEPD@stdout?3?5fflush?5failed?5?9?5err?$DN?$CFd?5@ 0000000180003660     libJNIreferences.obj
 0002:00000690       ??_C@_0CO@KBGKJPBD@stderr?3?5fflush?5failed?5?9?5err?$DN?$CFd?5@ 0000000180003690     libJNIreferences.obj
 0002:000006d0       _pDefaultRawDllMain        00000001800036d0     MSVCRT:dll_dllmain.obj
 0002:000006d0       _pRawDllMain               00000001800036d0     MSVCRT:dll_dllmain.obj
 0002:000006e0       __xmm@ffffffffffffffffffffffffffffffff 00000001800036e0     MSVCRT:utility.obj
 0002:000006f0       _load_config_used          00000001800036f0     MSVCRT:loadcfg.obj
 0002:00000900       __volatile_metadata        0000000180003900     <linker-defined>
 0002:00000c00       __rtc_iaa                  0000000180003c00     MSVCRT:initsect.obj
 0002:00000c08       __rtc_izz                  0000000180003c08     MSVCRT:initsect.obj
 0002:00000c10       __rtc_taa                  0000000180003c10     MSVCRT:initsect.obj
 0002:00000c18       __rtc_tzz                  0000000180003c18     MSVCRT:initsect.obj
 0002:00000fc0       __IMPORT_DESCRIPTOR_KERNEL32 0000000180003fc0     kernel32:KERNEL32.dll
 0002:00000fd4       __IMPORT_DESCRIPTOR_VCRUNTIME140 0000000180003fd4     vcruntime:VCRUNTIME140.dll
 0002:00000fe8       __IMPORT_DESCRIPTOR_api-ms-win-crt-stdio-l1-1-0 0000000180003fe8     ucrt:api-ms-win-crt-stdio-l1-1-0.dll
 0002:00000ffc       __IMPORT_DESCRIPTOR_api-ms-win-crt-heap-l1-1-0 0000000180003ffc     ucrt:api-ms-win-crt-heap-l1-1-0.dll
 0002:00001010       __IMPORT_DESCRIPTOR_api-ms-win-crt-runtime-l1-1-0 0000000180004010     ucrt:api-ms-win-crt-runtime-l1-1-0.dll
 0002:00001024       __IMPORT_DESCRIPTOR_api-ms-win-crt-string-l1-1-0 0000000180004024     ucrt:api-ms-win-crt-string-l1-1-0.dll
 0002:00001038       __NULL_IMPORT_DESCRIPTOR   0000000180004038     kernel32:KERNEL32.dll
 0003:00000000       __security_cookie          0000000180005000     MSVCRT:gs_cookie.obj
 0003:00000008       __security_cookie_complement 0000000180005008     MSVCRT:gs_cookie.obj
 0003:00000010       __scrt_native_dllmain_reason 0000000180005010     MSVCRT:utility.obj
 0003:00000018       __isa_available            0000000180005018     MSVCRT:cpu_disp.obj
 0003:0000001c       __isa_enabled              000000018000501c     MSVCRT:cpu_disp.obj
 0003:00000020       __memset_fast_string_threshold 0000000180005020     MSVCRT:cpu_disp.obj
 0003:00000028       __memset_nt_threshold      0000000180005028     MSVCRT:cpu_disp.obj
 0003:00000030       __scrt_ucrt_dll_is_in_use  0000000180005030     MSVCRT:ucrt_stubs.obj
 0003:00000040       ?_OptionsStorage@?1??__local_stdio_printf_options@@9@4_KA 0000000180005040     libJNIreferences.obj
 0003:000005f0       ?__type_info_root_node@@3U__type_info_node@@A 00000001800055f0     MSVCRT:tncleanup.obj
 0003:00000600       ?_OptionsStorage@?1??__local_stdio_scanf_options@@9@4_KA 0000000180005600     MSVCRT:default_local_stdio_options.obj
 0003:00000608       __scrt_current_native_startup_state 0000000180005608     MSVCRT:utility.obj
 0003:00000610       __scrt_native_startup_lock 0000000180005610     MSVCRT:utility.obj
 0003:00000650       __scrt_debugger_hook_flag  0000000180005650     MSVCRT:utility_desktop.obj
 0003:00000654       __favor                    0000000180005654     MSVCRT:cpu_disp.obj
 0003:00000658       __dyn_tls_init_callback    0000000180005658     <common>

 entry point at        0001:00000dc0

 Static symbols

 0000:ffff8000       .debug$S                   0000000180000000     JNIreferences.exp
 0000:ffff8000       .debug$S                   0000000180000000     vcruntime:VCRUNTIME140.dll
 0000:ffff8000       .debug$S                   0000000180000000     vcruntime:VCRUNTIME140.dll
 0000:ffff8000       .debug$S                   0000000180000000     vcruntime:VCRUNTIME140.dll
 0000:ffff8000       .debug$S                   0000000180000000     vcruntime:VCRUNTIME140.dll
 0000:ffff8000       .debug$S                   0000000180000000     vcruntime:VCRUNTIME140.dll
 0000:ffff8000       .debug$S                   0000000180000000     vcruntime:VCRUNTIME140.dll
 0000:ffff8000       .debug$S                   0000000180000000     vcruntime:VCRUNTIME140.dll
 0000:ffff8000       .debug$S                   0000000180000000     ucrt:api-ms-win-crt-heap-l1-1-0.dll
 0000:ffff8000       .debug$S                   0000000180000000     ucrt:api-ms-win-crt-runtime-l1-1-0.dll
 0000:ffff8000       .debug$S                   0000000180000000     ucrt:api-ms-win-crt-runtime-l1-1-0.dll
 0000:ffff8000       .debug$S                   0000000180000000     ucrt:api-ms-win-crt-runtime-l1-1-0.dll
 0000:ffff8000       .debug$S                   0000000180000000     ucrt:api-ms-win-crt-runtime-l1-1-0.dll
 0000:ffff8000       .debug$S                   0000000180000000     ucrt:api-ms-win-crt-runtime-l1-1-0.dll
 0000:ffff8000       .debug$S                   0000000180000000     ucrt:api-ms-win-crt-runtime-l1-1-0.dll
 0000:ffff8000       .debug$S                   0000000180000000     ucrt:api-ms-win-crt-runtime-l1-1-0.dll
 0000:ffff8000       .debug$S                   0000000180000000     ucrt:api-ms-win-crt-runtime-l1-1-0.dll
 0000:ffff8000       .debug$S                   0000000180000000     ucrt:api-ms-win-crt-runtime-l1-1-0.dll
 0000:ffff8000       .debug$S                   0000000180000000     ucrt:api-ms-win-crt-runtime-l1-1-0.dll
 0000:ffff8000       .debug$S                   0000000180000000     ucrt:api-ms-win-crt-runtime-l1-1-0.dll
 0000:ffff8000       .debug$S                   0000000180000000     ucrt:api-ms-win-crt-runtime-l1-1-0.dll
 0000:ffff8000       .debug$S                   0000000180000000     ucrt:api-ms-win-crt-runtime-l1-1-0.dll
 0000:ffff8000       .debug$S                   0000000180000000     ucrt:api-ms-win-crt-stdio-l1-1-0.dll
 0000:ffff8000       .debug$S                   0000000180000000     ucrt:api-ms-win-crt-stdio-l1-1-0.dll
 0000:ffff8000       .debug$S                   0000000180000000     ucrt:api-ms-win-crt-stdio-l1-1-0.dll
 0000:ffff8000       .debug$S                   0000000180000000     ucrt:api-ms-win-crt-stdio-l1-1-0.dll
 0000:ffff8000       .debug$S                   0000000180000000     ucrt:api-ms-win-crt-string-l1-1-0.dll
 0000:ffff8000       .debug$S                   0000000180000000     ucrt:api-ms-win-crt-string-l1-1-0.dll
 0000:ffff8000       .debug$S                   0000000180000000     ucrt:api-ms-win-crt-string-l1-1-0.dll
 0000:ffff8000       .debug$S                   0000000180000000     ucrt:api-ms-win-crt-string-l1-1-0.dll
 0000:ffff8000       .debug$S                   0000000180000000     kernel32:KERNEL32.dll
 0000:ffff8000       .debug$S                   0000000180000000     kernel32:KERNEL32.dll
 0000:ffff8000       .debug$S                   0000000180000000     kernel32:KERNEL32.dll
 0000:ffff8000       .debug$S                   0000000180000000     kernel32:KERNEL32.dll
 0000:ffff8000       .debug$S                   0000000180000000     kernel32:KERNEL32.dll
 0000:ffff8000       .debug$S                   0000000180000000     kernel32:KERNEL32.dll
 0000:ffff8000       .debug$S                   0000000180000000     kernel32:KERNEL32.dll
 0000:ffff8000       .debug$S                   0000000180000000     kernel32:KERNEL32.dll
 0000:ffff8000       .debug$S                   0000000180000000     kernel32:KERNEL32.dll
 0000:ffff8000       .debug$S                   0000000180000000     kernel32:KERNEL32.dll
 0000:ffff8000       .debug$S                   0000000180000000     kernel32:KERNEL32.dll
 0000:ffff8000       .debug$S                   0000000180000000     kernel32:KERNEL32.dll
 0000:ffff8000       .debug$S                   0000000180000000     kernel32:KERNEL32.dll
 0000:ffff8000       .debug$S                   0000000180000000     kernel32:KERNEL32.dll
 0000:ffff8000       .debug$S                   0000000180000000     kernel32:KERNEL32.dll
 0000:ffff8000       .debug$S                   0000000180000000     kernel32:KERNEL32.dll
 0000:ffff8000       .debug$S                   0000000180000000     kernel32:KERNEL32.dll
 0001:00000500       file_basename              0000000180001500 f   libJNIreferences.obj
 0001:00000980       capture_previous_context   0000000180001980 f   MSVCRT:gs_report.obj
 0001:00000a70       $$000000                   0000000180001a70     MSVCRT:amdsecgs.obj
 0001:00000aa0       ?dllmain_crt_dispatch@@YAHQEAUHINSTANCE__@@KQEAX@Z 0000000180001aa0 f   MSVCRT:dll_dllmain.obj
 0001:00000af0       ?dllmain_crt_process_attach@@YAHQEAUHINSTANCE__@@QEAX@Z 0000000180001af0 f   MSVCRT:dll_dllmain.obj
 0001:00000c08       ?dllmain_crt_process_detach@@YAH_N@Z 0000000180001c08 f   MSVCRT:dll_dllmain.obj
 0001:00000c8c       ?dllmain_dispatch@@YAHQEAUHINSTANCE__@@KQEAX@Z 0000000180001c8c f   MSVCRT:dll_dllmain.obj
 0001:00001640       $$000000                   0000000180002640     MSVCRT:guard_dispatch.obj
 0001:00001660       $$000000                   0000000180002660     MSVCRT:guard_xfg_dispatch.obj
 0001:00001676       ?fin$0@?0??dllmain_crt_process_attach@@YAHQEAUHINSTANCE__@@QEAX@Z@4HA 0000000180002676 f   MSVCRT:dll_dllmain.obj
 0001:0000168d       ?fin$0@?0??dllmain_crt_process_detach@@YAH_N@Z@4HA 000000018000268d f   MSVCRT:dll_dllmain.obj
 0001:000016a6       ?fin$1@?0??dllmain_crt_process_detach@@YAH_N@Z@4HA 00000001800026a6 f   MSVCRT:dll_dllmain.obj
 0001:000016ba       ?filt$0@?0??dllmain_dispatch@@YAHQEAUHINSTANCE__@@KQEAX@Z@4HA 00000001800026ba f   MSVCRT:dll_dllmain.obj
 0001:000016f0       __scrt_is_nonwritable_in_current_image$filt$0 00000001800026f0 f   MSVCRT:utility.obj
 0002:000006c0       GS_ExceptionPointers       00000001800036c0     MSVCRT:gs_report.obj
 0002:00000c20       $unwind$fprintf            0000000180003c20     libJNIreferences.obj
 0002:00000c2c       $unwind$printf             0000000180003c2c     libJNIreferences.obj
 0002:00000c38       $unwind$?CallVoidMethod@JNIEnv_@@QEAAXPEAV_jobject@@PEAU_jmethodID@@ZZ 0000000180003c38     libJNIreferences.obj
 0002:00000c38       $unwind$nsk_lcomplain      0000000180003c38     libJNIreferences.obj
 0002:00000c40       $unwind$nsk_lvcomplain     0000000180003c40     libJNIreferences.obj
 0002:00000c58       $unwind$nsk_vprintf        0000000180003c58     libJNIreferences.obj
 0002:00000c68       $unwind$nsk_printf         0000000180003c68     libJNIreferences.obj
 0002:00000c70       $unwind$Java_nsk_share_ReferringObject_createJNIGlobalReferenceNative 0000000180003c70     libJNIreferences.obj
 0002:00000c70       $unwind$Java_nsk_share_ReferringObject_createJNIWeakReferenceNative 0000000180003c70     libJNIreferences.obj
 0002:00000c88       $unwind$Java_nsk_share_ReferringObject_createJNILocalReferenceNative 0000000180003c88     libJNIreferences.obj
 0002:00000c88       $unwind$Java_nsk_share_ReferringObject_deleteJNIGlobalReferenceNative 0000000180003c88     libJNIreferences.obj
 0002:00000c88       $unwind$Java_nsk_share_ReferringObject_deleteJNIWeakReferenceNative 0000000180003c88     libJNIreferences.obj
 0002:00000c88       $unwind$_DllMainCRTStartup 0000000180003c88     MSVCRT:dll_dllmain.obj
 0002:00000c98       $unwind$__report_gsfailure 0000000180003c98     MSVCRT:gs_report.obj
 0002:00000ca0       $unwind$capture_previous_context 0000000180003ca0     MSVCRT:gs_report.obj
 0002:00000cac       $unwind$__raise_securityfailure 0000000180003cac     MSVCRT:gs_report.obj
 0002:00000cac       $unwind$__scrt_initialize_crt 0000000180003cac     MSVCRT:utility.obj
 0002:00000cac       $unwind$__scrt_initialize_onexit_tables 0000000180003cac     MSVCRT:utility.obj
 0002:00000cac       $unwind$__scrt_release_startup_lock 0000000180003cac     MSVCRT:utility.obj
 0002:00000cac       $unwind$__scrt_uninitialize_crt 0000000180003cac     MSVCRT:utility.obj
 0002:00000cb4       $unwind$__GSHandlerCheckCommon 0000000180003cb4     MSVCRT:gshandler.obj
 0002:00000cbc       $unwind$__scrt_initialize_default_local_stdio_options 0000000180003cbc     MSVCRT:default_local_stdio_options.obj
 0002:00000cbc       $unwind$?dllmain_crt_dispatch@@YAHQEAUHINSTANCE__@@KQEAX@Z 0000000180003cbc     MSVCRT:dll_dllmain.obj
 0002:00000cbc       $unwind$DllMain            0000000180003cbc     MSVCRT:dll_dllmain_stub.obj
 0002:00000cbc       $unwind$__GSHandlerCheck   0000000180003cbc     MSVCRT:gshandler.obj
 0002:00000cbc       $unwind$__scrt_acquire_startup_lock 0000000180003cbc     MSVCRT:utility.obj
 0002:00000cbc       $unwind$__scrt_dllmain_after_initialize_c 0000000180003cbc     MSVCRT:utility.obj
 0002:00000cbc       $unwind$__scrt_dllmain_before_initialize_c 0000000180003cbc     MSVCRT:utility.obj
 0002:00000cbc       $unwind$__scrt_dllmain_crt_thread_attach 0000000180003cbc     MSVCRT:utility.obj
 0002:00000cbc       $unwind$__scrt_dllmain_crt_thread_detach 0000000180003cbc     MSVCRT:utility.obj
 0002:00000cbc       $unwind$__scrt_dllmain_uninitialize_c 0000000180003cbc     MSVCRT:utility.obj
 0002:00000cbc       $unwind$__scrt_dllmain_uninitialize_critical 0000000180003cbc     MSVCRT:utility.obj
 0002:00000cc8       $xdatasym                  0000000180003cc8     MSVCRT:amdsecgs.obj
 0002:00000ccc       $unwind$?dllmain_crt_process_attach@@YAHQEAUHINSTANCE__@@QEAX@Z 0000000180003ccc     MSVCRT:dll_dllmain.obj
 0002:00000d08       $unwind$?fin$0@?0??dllmain_crt_process_attach@@YAHQEAUHINSTANCE__@@QEAX@Z@4HA 0000000180003d08     MSVCRT:dll_dllmain.obj
 0002:00000d08       $unwind$?fin$0@?0??dllmain_crt_process_detach@@YAH_N@Z@4HA 0000000180003d08     MSVCRT:dll_dllmain.obj
 0002:00000d08       $unwind$?fin$1@?0??dllmain_crt_process_detach@@YAH_N@Z@4HA 0000000180003d08     MSVCRT:dll_dllmain.obj
 0002:00000d10       $unwind$?dllmain_crt_process_detach@@YAH_N@Z 0000000180003d10     MSVCRT:dll_dllmain.obj
 0002:00000d64       $unwind$?dllmain_dispatch@@YAHQEAUHINSTANCE__@@KQEAX@Z 0000000180003d64     MSVCRT:dll_dllmain.obj
 0002:00000d8c       $unwind$?filt$0@?0??dllmain_dispatch@@YAHQEAUHINSTANCE__@@KQEAX@Z@4HA 0000000180003d8c     MSVCRT:dll_dllmain.obj
 0002:00000d94       $unwind$__security_init_cookie 0000000180003d94     MSVCRT:gs_support.obj
 0002:00000da0       $unwind$__scrt_is_nonwritable_in_current_image 0000000180003da0     MSVCRT:utility.obj
 0002:00000dc0       $unwind$__scrt_is_nonwritable_in_current_image$filt$0 0000000180003dc0     MSVCRT:utility.obj
 0002:00000dc8       $unwind$__scrt_dllmain_exception_filter 0000000180003dc8     MSVCRT:utility.obj
 0002:00000ddc       $unwind$__scrt_fastfail    0000000180003ddc     MSVCRT:utility_desktop.obj
 0002:00000dec       $unwind$_RTC_Initialize    0000000180003dec     MSVCRT:initsect.obj
 0002:00000dec       $unwind$_RTC_Terminate     0000000180003dec     MSVCRT:initsect.obj
 0002:00000df8       $unwind$__isa_available_init 0000000180003df8     MSVCRT:cpu_disp.obj
 0002:00000e08       $xdatasym                  0000000180003e08     MSVCRT:guard_dispatch.obj
 0002:00000e10       $xdatasym                  0000000180003e10     MSVCRT:guard_xfg_dispatch.obj
 0002:00000e20       .edata                     0000000180003e20     JNIreferences.exp
 0002:00000e48       rgpv                       0000000180003e48     JNIreferences.exp
 0002:00000e5c       rgszName                   0000000180003e5c     JNIreferences.exp
 0002:00000e70       rgwOrd                     0000000180003e70     JNIreferences.exp
 0002:00000e7a       szName                     0000000180003e7a     JNIreferences.exp
 0002:00000e8c       $N00001                    0000000180003e8c     JNIreferences.exp
 0002:00000eca       $N00002                    0000000180003eca     JNIreferences.exp
 0002:00000f07       $N00003                    0000000180003f07     JNIreferences.exp
 0002:00000f43       $N00004                    0000000180003f43     JNIreferences.exp
 0002:00000f81       $N00005                    0000000180003f81     JNIreferences.exp
 0002:00001306       .idata$6                   0000000180004306     kernel32:KERNEL32.dll
 0002:00001360       .idata$6                   0000000180004360     vcruntime:VCRUNTIME140.dll
 0002:00001490       .idata$6                   0000000180004490     ucrt:api-ms-win-crt-stdio-l1-1-0.dll
 0002:000014b0       .idata$6                   00000001800044b0     ucrt:api-ms-win-crt-heap-l1-1-0.dll
 0002:000014d0       .idata$6                   00000001800044d0     ucrt:api-ms-win-crt-runtime-l1-1-0.dll
 0002:000014f2       .idata$6                   00000001800044f2     ucrt:api-ms-win-crt-string-l1-1-0.dll
 0003:00000048       globalReferences           0000000180005048     libJNIreferences.obj
 0003:00000050       weakReferences             0000000180005050     libJNIreferences.obj
 0003:00000058       nsk_context                0000000180005058     libJNIreferences.obj
 0003:00000070       GS_ExceptionRecord         0000000180005070     MSVCRT:gs_report.obj
 0003:00000110       GS_ContextRecord           0000000180005110     MSVCRT:gs_report.obj
 0003:000005e0       ?__proc_attached@@3HA      00000001800055e0     MSVCRT:dll_dllmain.obj
 0003:00000618       ?is_initialized_as_dll@@3_NA 0000000180005618     MSVCRT:utility.obj
 0003:00000619       ?module_local_atexit_table_initialized@@3_NA 0000000180005619     MSVCRT:utility.obj
 0003:00000620       ?module_local_atexit_table@@3U_onexit_table_t@@A 0000000180005620     MSVCRT:utility.obj
 0003:00000638       ?module_local_at_quick_exit_table@@3U_onexit_table_t@@A 0000000180005638     MSVCRT:utility.obj
